:100000000000000000000528090007309F0083164B
:100010009F01EB3086008A018312552882008207F7
:10002000063443346F346D346D346F346E3482076C
:100030000D340034013402340434083410341F34D5
:100040000F3417341B341D341E340034820704343B
:1000500044346F346E34653482070434463461347A
:1000600069346C348207033449346E347434820743
:10007000033449342F344F3482070C3449346E34FE
:100080004F3475347434313430345F34543465341F
:1000900073347434820704345434653473347434E0
:1000A000820703345234653467348C243D30DE00DB
:1000B00023258C24A80106169E244F08A50036256A
:1000C000362530302502031C75283A3025020318E6
:1000D00075282508DD001D25280DA900A90D290D6D
:1000E000F8392507D03EA800E92873302502031D02
:1000F00082282508DD001D258C242808D300C32470
:10010000A801E92877302502031DAE282508DD0067
:100110001D258C242808D300C324A801A70105307D
:10012000270203189E28BD245208A9002030270763
:100130008400290883138000A70A8F28A7010530AF
:1001400027020318AC2820302707840083130008F7
:10015000D000A424A70A9F288C24E928693025020E
:10016000031DBF282508DD001D258C24FD30D3008C
:10017000C324FF23FF23FF2309240924E928743023
:100180002502031DC9282508DD001D258C247921A1
:10019000E92863302502031DD6282508DD001D252A
:1001A0008C242808AA00EA20A801E928FC302502AE
:1001B0000319E9283C30DD001D252508D000A424C2
:1001C0003E30DD001D258C242808D000A4248C247A
:1001D000A8015B283B30B2002A083202B10002308D
:1001E000AC00FF30AD00F030AE005430DD001D2516
:1001F0000530D000A4243108D000A4248C2443303E
:10020000DD001D25FA30D300C324BD245208D000E0
:10021000A424FB30D300C324B001AF01861A0E29F9
:100220001129861A1729B00A0319AF0A1129483073
:10023000DD001D252F08D000A4244C30DD001D2535
:100240003008D000A42406302F0203184C290530B2
:100250002F02031C472930083102031C3F293108B3
:100260003002031C3729AB01AD01AE013E29F83045
:10027000AB003108B20030083202AD004629F93037
:10028000AB003008B20031083202AD004B29F83023
:10029000AB003108AD005329F930AB00FF30B2009C
:1002A00031083202AD004530DD001D252D08D0009B
:1002B000A4244D30DD001D252E08D000A4242D08D7
:1002C0002E02031D66298C24003474292E082D0269
:1002D000031C7129AC03031D7029AE0A0230AC0067
:1002E00074292D08AE00AD0A2B08D300C3248C243A
:1002F000FF287F231B245130DE0023254B30DE00F6
:1003000023258C24B901083039020318F82901305B
:100310008A003908820793299829B5299D29A2299D
:10032000A729AC29B1290230BA001230BB00B52987
:100330000430BA001430BB00B5290830BA001830B8
:10034000BB00B5290A30BA001A30BB00B5290C3001
:10035000BA001C30BB00B5290E30BA001E30BB00FD
:10036000B5291030BA00FF30BB001730D300C324CA
:10037000B601023036020318F629B8010D303802F2
:100380000318F429380A8A011720B7003B0A031919
:10039000CF293B083604D300C3243708D5293608B3
:1003A00003192030031D40303704D300C3243A081A
:1003B0003604D300C324BD245208BC0037020319FD
:1003C000F2293908D000A4243608D000A424370824
:1003D000D000A4243C08D000A4245130CD003030FB
:1003E000CE009324B80ABE29B60AB929B90A8329CE
:1003F0003830DE0023254B30DE0023258C24B60167
:10040000023036020318E72A3608031D122A143078
:10041000D300C3241530D300C3241530D300C32424
:100420000A301C2A1430D300C3240A30D300C3245A
:100430001530D300C3241530D300C324B4012030B9
:1004400034020318E52AB501B301341C292A3514F6
:10045000B514B41C2D2A3515B515341D312A3516A1
:100460003314B41D352AB3143315341E392AB31589
:10047000331620303504D300C32440303304D30076
:10048000C3240630D300C324BD245208BC00350267
:100490000319582A3408D000A4243508D000A42415
:1004A0003C08D000A4243830CD003130CE00932455
:1004B0000730D300C324BD245208BC003302031903
:1004C0006F2A3408D000A4243308D000A4243C08A8
:1004D000D000A4243830CD003230CE009324123026
:1004E000D300C3241F30D300C3241330D300C3244C
:1004F0001F30D300C324D301C324BD245208BC0041
:100500001F303C0635020319932A3408D000A42476
:100510003508D000A4243C08D000A4243830CD00F5
:100520003330CE0093240130D300C324BD245208BD
:10053000BC001F303C0633020319AC2A3408D0003B
:10054000A4243308D000A4243C08D000A4243830CC
:10055000CD003430CE0093241230D300C324D30115
:10056000C3241330D300C324D301C324D301C32431
:10057000BD245208BC0035020319CC2A3408D0002F
:10058000A4243508D000A4243C08D000A42438308A
:10059000CD003530CE0093240130D300C324BD24D8
:1005A0005208BC0033020319E32A3408D000A42403
:1005B0003308D000A4243C08D000A4243830CD0057
:1005C0003630CE009324B40A1F2AB60A002A3330EC
:1005D000DE0023254B30DE0023258C241430D3008D
:1005E000C3241530D300C3241530D300C3240A30EC
:1005F000D300C3241830BD002030BE001F30BF0020
:100600004030C00046231930BD004030BE001F30CE
:10061000BF004230C00046231A30BD002030BE006B
:10062000BF014430C00046231B30BD004030BE0037
:10063000BF014630C00046231C30BD002030BE0044
:10064000BF014830C00046231D30BD004030BE0011
:10065000BF014A30C00046231E30BD002030BE001E
:100660001F30BF004C30C00046231F30BD0040305B
:10067000BE001F30BF004E30C00046231730D300ED
:10068000C3242730DE0023258C2400343E083F0499
:10069000D300C3243D08D300C3241F30D300C32498
:1006A000EF30D300C324BD245208C1000319602BCE
:1006B0004108D000A4243330CD004008CE0093245C
:1006C0001F303F063E04D300C324EF30D300C324C1
:1006D000BD245208C10041030319762B4108D00004
:1006E000A4243330CD00400ACE0093243D08D3002B
:1006F000C324D301C324F030D300C3240034FD301D
:10070000D300C3240130C400C030C500F423C401A9
:10071000C130C500F4230D30C400C230C500F4233D
:10072000C401C330C500F423C401C430C500F423A0
:10073000C401C530C500F423C401C630C500F4238C
:10074000C401C730C500F4238C24FF23FF230924F0
:10075000092414244808FD30D300C3240130C40008
:10076000C830C500F423FE30D300C324BD24520892
:10077000C200FF30D300C324FF30D300C324FE30B7
:10078000D300C324BD245208C3000230430203191E
:10079000CE2B1030CD00C930CE009324FB30D300D7
:1007A000C324BD2452080319DA2B1030CD00CA30FF
:1007B000CE009324FA30D300C324BD245208C200D3
:1007C000F930D300C324F830D300C324FA30D30067
:1007D000C324BD24520842020319F32B1030CD006C
:1007E000CB30CE009324003414244808440203196B
:1007F000FE2B1030CD004508CE0093240034083085
:10080000C60014244808D000A424C60B012C8C2454
:10081000003414244808C70014244808DD001D25AE
:10082000C70B0C2C8C240034FC30D300C324BD2413
:100830005208C8000034F030D300C324CA01D030BD
:10084000CB007A24F530D300C3240130CA00D13064
:10085000CB007A24F430D300C324CA01D230CB00B9
:100860007A24F130D300C3240130CA00D330CB0046
:100870007A24F030D300C324CA01D430CB007A24C8
:10088000F730D300C3240230CA00D530CB007A241D
:10089000F630D300C324CA01D630CB007A24F2301C
:1008A000D300C3240230CA00D730CB007A24F03002
:1008B000D300C324CA01D830CB007A24F330D3004C
:1008C000C3240330C9003625C90B632C861E6D2C4A
:1008D0003330CD00D930CE0093240130CA00DA3055
:1008E000CB007A24F030D300C324CA01DB30CB0024
:1008F0007A240034EF30D300C324BD245208CC0046
:100900004A0203198B2C4C08D000A4243330CD00AC
:100910004B08CE00932400340D30DD001D250A3035
:10092000DD001D2500342D30DE0023254D08DE00BE
:1009300023254E08D000A4248C2400340230D40097
:10094000C9245508CF000034500ED100D10C510CF1
:100950000339303EDD001D25500CD100D10C510C67
:100960000739303EDD001D2507305005303EDD00E3
:100970001D252030DD001D2500342030D400C92481
:100980005508D20000345308D9001030DA00F7249B
:100990000034D601060854050319D72CD60356088F
:1009A000031DD52CFC30D50000343625CA2C362545
:1009B00036253625D7010230D800D80BDD2C0000B3
:1009C00000000830D60036250310D70C0608540561
:1009D000031DD71736253625000000000000000053
:1009E000D60BE32C362536255708D5000034FF30CA
:1009F0005A06DC0086003625362536250000000024
:100A000000000000000000000830DB005918FF3033
:100A1000591C5C0886000310D90C3625362536256E
:100A200000000000DB0B062D0000FF30860036259D
:100A3000362536250000000000345D08D90004305A
:100A4000DA00F7240034E0018A015E080E2060021B
:100A50000318322D600A5E078A010E20DD001D2575
:100A6000E00A242D2030DD001D2500347030E10027
:0A0A7000E10B382D000000000034F7
:02400E00293F48
:00000001FF
